S025000062696E2F64656D6F70726F675F6F6C696D65785F73746D3332703430352E737265632C
S3150800800000000220FD8500084D8600084D86000800
S315080080104D8600084D8600084D86000800000000C1
S315080080200000000000000000000000004D86000867
S315080080304D860008000000004D86000835990008A6
S315080080404D8600084D8600084D8600084D860008B6
S315080080504D8600084D8600084D8600084D860008A6
S315080080604D8600084D8600084D8600084D86000896
S315080080704D8600084D8600084D8600084D86000886
S315080080804D8600084D8600084D8600084D86000876
S315080080904D8600084D8600084D8600084D86000866
S315080080A04D8600084D8600084D8600084D86000856
S315080080B04D8600084D8600084D8600084D86000846
S315080080C04D8600084D8600084D8600084D86000836
S315080080D04D8600084D8600084D8600084D86000826
S315080080E04D8600084D8600084D8600084D86000816
S315080080F04D8600084D8600084D8600084D86000806
S315080081004D8600084D8600084D8600084D860008F5
S315080081104D8600084D8600084D8600084D860008E5
S315080081204D8600084D8600084D8600084D860008D5
S315080081304D86000800000000000000004D8600087B
S315080081404D8600084D8600084D8600084D860008B5
S315080081504D8600084D8600084D8600084D860008A5
S315080081604D8600084D8600084D8600084D86000895
S315080081704D8600084D86000800000000000000003B
S311080081804D8600084D860008EE11AA5531
S3150800818C10B5054C237833B9044B13B10448AFF337
S3150800819C00800123237010BD380400200000000065
S315080081AC289E000808B5034B1BB103490348AFF3D7
S315080081BC008008BD000000003C040020289E000832
S315080081CC53B94AB9002908BF00281CBF4FF0FF3124
S315080081DC4FF0FF3000F074B9ADF1080C6DE904CE20
S315080081EC00F006F8DDF804E0DDE9022304B0704778
S315080081FC2DE9F047089E04468846002B40F08580FA
S3150800820C8A42154648D9B2FA82F24AB1C2F1200717
S3150800821C01FA02F320FA07F7954047EA0308944057
S3150800822C4FEA154E230CB8FBFEF71FFA85FC0EFB1E
S3150800823C178843EA084307FB0CF1994209D9EB184E
S3150800824C07F1FF3080F0E380994240F2E080023F6C
S3150800825C2B445B1AA4B2B3FBFEF00EFB103344EAB4
S3150800826C034400FB0CFCA44509D92C1900F1FF3377
S3150800827C80F0CB80A44540F2C88002382C4440EAF2
S3150800828C0740A4EB0C0400271EB1D4400023C6E912
S3150800829C00433946BDE8F087002A53D0B2FA82F279
S315080082AC002A40F0B680491B4FEA154E1FFA85F88E
S315080082BC0127B1FBFEFC230C0EFB1C1143EA014300
S315080082CC08FB0CF1994207D9EB180CF1FF3002D2D6
S315080082DC994200F2EC808446591AA3B2B1FBFEF01F
S315080082EC0EFB101443EA044408FB00F8A04507D912
S315080082FC2C1900F1FF3302D2A04500F2DC80184697
S3150800830CA4EB080440EA0C40BEE78B4208D9002EC1
S3150800831C78D00027C6E9000138463946BDE8F0870B
S3150800832CB3FA83F77FB98B4202D3824200F2BD803F
S3150800833C841A61EB030301209846002EA9D0C6E9DE
S3150800834C0048A6E7FFDEC7F12005BB4022FA05FC6C
S3150800835C4CEA030C01FA07F420FA05F821FA05F39E
S3150800836C4FEA1C4E48EA0404B3FBFEF9210C0EFB3B
S3150800837C19331FFA8CF841EA034309FB08FA9A45A4
S3150800838C02FA07F200FA07F10BD91CEB030309F101
S3150800839CFF3080F088809A4540F28580A9F1020961
S315080083AC6344A3EB0A03A4B2B3FBFEF00EFB103333
S315080083BC44EA034400FB08F8A04508D91CEB04045E
S315080083CC00F1FF336BD2A04569D90238644440EA00
S315080083DC0940A4EB0804A0FB02894C45C6464B464B
S315080083EC54D351D0002E69D0B1EB0E0264EB0304C2
S315080083FC04FA05F522FA07F3FC401D43C6E90054B6
S3150800840C002746E73746304643E7184637E7074618
S3150800841C1FE7C2F1200320FA03F7954001FA02F090
S3150800842C21FA03F34FEA154E3843010CB3FBFEF75A
S3150800843C1FFA85F80EFB173341EA034107FB08F3CD
S3150800844C8B4204FA02F407D9691807F1FF3C28D2C3
S3150800845C8B4226D9023F2944CB1A81B2B3FBFEF0D4
S3150800846C0EFB103341EA034100FB08F38B4207D994
S3150800847C691800F1FF3C10D28B420ED902382944F8
S3150800848CC91A40EA074714E74145ABD2B8EB020EC6
S3150800849C69EB0C0201381346A4E76046F0E7184668
S315080084AC95E76746D8E781467BE7384645E7ACF15A
S315080084BC020C2B4410E702382C4421E73746E8E631
S315080084CC704700BF70B50D4E0D4D761BB61006D015
S315080084DC0024013455F8043B9847A642F9D1094EB5
S315080084EC094D761B01F09AFCB61006D0002401340F
S315080084FC55F8043B9847A642F9D170BD889E0008EA
S3150800850C889E0008909E0008889E0008024B13B1AE
S3150800851C024800F005B870470000000039850008CD
S3150800852C002301461A46184600F01EB838B50A4C00
S3150800853C0A4D641BA4100AD004F18043013B05EBD9
S3150800854C8305013C55F804399847002CF9D1BDE848
S3150800855C384001F069BC00BF949E0008909E000844
S3150800856C704700BF704700BF2DE9F0411E4C054609
S3150800857C206890461F460E46FFF7F2FF1B4B1A68FB
S3150800858CD2F8483133B35A6820681F2A27DC4DB90C
S3150800859C911C01325A6043F82160FFF7E3FF002073
S315080085ACBDE8F08103EB82010124C1F8888004FA46
S315080085BC02FED3F88841022D44EA0E0CC3F888C192
S315080085CCC1F80871E4D1D3F88C114EEA0104C3F84A
S315080085DC8C41DDE702F5A673C2F84831D3E7FFF7FD
S315080085ECC1FF4FF0FF30DBE728040020409E00084F
S315080085FCDFF834D0002103E00C4B5B5843500431B0
S3150800860C0B480C4B42189A42F6D30B4A02E000234D
S3150800861C42F8043B094B9A42F9D300F013F8FFF7DA
S3150800862C51FF01F019FA704700000220949E0008C9
S3150800863C00000020380400203804002034050020EF
S3150800864CFEE700000F49D1F8883043F47003C1F8EF
S3150800865C88300D4B1A6842F001021A6000209860A7
S3150800866C1A6822F0847222F480321A60074A5A6019
S3150800867C1A6822F480221A60D8604FF000638B6067
S3150800868C704700BF00ED00E00038024010300024AF
S3150800869C002800F0B98170B582B00446036813F05F
S315080086AC010F3BD0A64B9B6803F00C03042B2CD074
S315080086BCA34B9B6803F00C03082B21D06368B3F516
S315080086CC803F4FD0B3F5A02F52D09D4B1A6822F499
S315080086DC80321A601A6822F480221A606368002BAA
S315080086EC50D001F001F90546954B1B6813F4003F71
S315080086FC14D101F0F9F8401B6428F5D903208AE156
S3150800870C8F4B5B6813F4800FD8D08D4B1B6813F412
S3150800871C003F03D06368002B00F07881236813F0C0
S3150800872C020F54D0864B9B6813F00C0F3ED0844B2B
S3150800873C9B6803F00C03082B33D0E368002B67D037
S3150800874C804B01221A6001F0CFF805467C4B1B685A
S3150800875C13F0020F53D101F0C7F8401B0228F5D9C4
S3150800876C032058E1764A136843F480331360B5E75F
S3150800877C734B1A6842F480221A601A6842F48032E3
S3150800878C1A60ABE701F0B0F805466D4B1B6813F49D
S3150800879C003FC3D001F0A8F8401B6428F5D9032084
S315080087AC39E1674B5B6813F4800FC6D1644B1B68C1
S315080087BC13F0020F03D0E368012B40F02981604ABD
S315080087CC136823F0F803216943EAC103136023688D
S315080087DC13F0080F40D0636963B35B4B01221A6030
S315080087EC01F082F80546564B5B6F13F0020F33D136
S315080087FC01F07AF8401B0228F5D903200BE1504A00
S3150800880C136823F0F803216943EAC1031360DEE712
S3150800881C4C4B00221A6001F067F80546484B1B685A
S3150800882C13F0020FD3D001F05FF8401B0228F5D9DC
S3150800883C0320F0E0444B00221A6001F055F8054677
S3150800884C3F4B5B6F13F0020F06D001F04DF8401B3F
S3150800885C0228F5D90320DEE0236813F0040F78D03C
S3150800886C374B1B6C13F0805F33D100230193344BC9
S3150800887C1A6C42F080521A641B6C03F080530193F5
S3150800888C019B0125314B1B6813F4807F23D0A36809
S3150800889C012B34D0052B38D0294B1A6F22F0010244
S315080088AC1A671A6F22F004021A67A368002B36D0CF
S315080088BC01F01AF80646224B1B6F13F0020F47D12C
S315080088CC01F012F8801B41F288339842F3D9032041
S315080088DCA1E00025D6E71D4A136843F4807313609C
S315080088EC01F002F80646194B1B6813F4807FCED1AB
S315080088FC00F0FAFF801B0228F5D903208BE0104AFA
S3150800890C136F43F001031367CFE70D4B1A6F42F051
S3150800891C04021A671A6F42F001021A67C5E700F0DB
S3150800892CE3FF0646064B1B6F13F0020F10D000F040
S3150800893CDBFF801B41F288339842F3D903206AE0A7
S3150800894C0038024000004742800E47420070004043
S3150800895CE5B9A369002B5DD0314A926802F00C0286
S3150800896C082A5AD0022B17D02E4B00221A6000F078
S3150800897CBBFF04462A4B1B6813F0007F42D000F05D
S3150800898CB3FF001B0228F5D9032044E0244A136CD4
S3150800899C23F080531364DCE7224B00221A6000F0A4
S315080089ACA3FF05461E4B1B6813F0007F06D000F08C
S315080089BC9BFF401B0228F5D903202CE0E369226AA9
S315080089CC1343626A43EA8213A26A5208013A43EADB
S315080089DC0243E26A43EA0263114A5360114B0122CD
S315080089EC1A6000F081FF04460D4B1B6813F0007FDC
S315080089FC06D100F079FF001B0228F5D903200AE0FE
S31508008A0C002008E0002006E001207047012002E063
S31508008A1C012000E0002002B070BD0120FBE700BF7A
S31508008A2C0038024060004742314B9B6803F00C0348
S31508008A3C042B58D0082B58D170B52D4B5A6802F018
S31508008A4C3F025B6813F4800F2AD0294B5868C0F391
S31508008A5C88100546002643011B1A66EB0604A1017D
S31508008A6C41EA93619801C01A61EB0401CB0043EA11
S31508008A7C5073C4001946601946EB01014B0243EAD0
S31508008A8CD0534402204619463346FFF799FB184B38
S31508008A9C5B68C3F3014301335B00B0FBF3F070BDB5
S31508008AAC134B5868C0F388100546002643011B1A59
S31508008ABC66EB0604A10141EA93619801C01A61EBC1
S31508008ACC0401CB0043EA5073C4001946601946EBFF
S31508008ADC01018B0243EA9053840220461946334619
S31508008AECFFF76EFBD3E7034870470348704700BF90
S31508008AFC0038024000127A000024F400002800F026
S31508008B0C9A8070B50446504B1B6803F00F038B42D2
S31508008B1C08D2CBB24C4A1370136803F00F038B427E
S31508008B2C40F08B80236813F0020F17D013F0040F54
S31508008B3C04D0464A936843F4E0539360236813F0D1
S31508008B4C080F04D0414A936843F4604393603F4A44
S31508008B5C936823F0F003A068034393600D462368DB
S31508008B6C13F0010F32D06368012B21D09A1E012A0B
S31508008B7C25D9364A126812F0020F60D033498A6832
S31508008B8C22F0030213438B6000F0AEFE06462F4B11
S31508008B9C9B6803F00C036268B3EB820F16D000F0E7
S31508008BACA3FE801B41F288339842F0D9032041E09A
S31508008BBC264A126812F4003FE0D101203AE0234A13
S31508008BCC126812F0007FD9D1012033E01E4B1B68C6
S31508008BDC03F00F03AB4207D9EAB21B4B1A701B689A
S31508008BEC03F00F03AB422CD1236813F0040F06D005
S31508008BFC164A936823F4E053E1680B4393602368A1
S31508008C0C13F0080F07D0114A936823F460432169BF
S31508008C1C43EAC1039360FFF707FF0C4B9B68C3F34A
S31508008C2C03130B4AD35CD8400A4B1860002000F09B
S31508008C3C0FFE002070BD012070470120FAE70120C5
S31508008C4CF8E70120F6E700BF003C02400038024076
S31508008C5C449E00082C040020014B1868704700BF7E
S31508008C6C2C04002008B5FFF7F7FF044B9B68C3F3E9
S31508008C7C8223034AD35CD84008BD00BF00380240A3
S31508008C8C549E000808B5FFF7E7FF044B9B68C3F32F
S31508008C9C4233034AD35CD84008BD00BF00380240B3
S31508008CAC549E00087047002800F0A18038B5044689
S31508008CBC90F82030D3B12268136823F002031360AE
S31508008CCC00F012FE054623685A6812F0020F10D0FF
S31508008CDC00F00AFE401B0A28F5D9636A43F40033F0
S31508008CEC6362052384F82030012038BDFFF7DAFFCC
S31508008CFCE1E71A6842F001021A6000F0F5FD054634
S31508008D0C23685A6812F0010F0DD100F0EDFD401BD7
S31508008D1C0A28F5D9636A43F400336362052384F899
S31508008D2C20300120E1E7227E012A3DD01A6822F084
S31508008D3C80021A60637E012B3BD02268136823F0ED
S31508008D4C40031360A37E012B39D02268136823F0E5
S31508008D5C20031360E37E012B37D02268136843F097
S31508008D6C10031360237F012B35D02268136823F078
S31508008D7C08031360637F012B33D02268136823F032
S31508008D8C04031360A368E2681343226913436269F8
S31508008D9C13436268013A21681343CB610020606271
S31508008DAC012384F82030A0E71A6842F080021A6082
S31508008DBCC0E72268136843F040031360C2E72268D1
S31508008DCC136843F020031360C4E72268136823F082
S31508008DDC10031360C6E72268136843F00803136090
S31508008DECC8E72268136843F004031360CAE7012036
S31508008DFC7047000090F82030DBB2012B0AD090F8AF
S31508008E0C2030DBB2022B05D0436A43F4802343623D
S31508008E1C0120704770B4424BD3F8002242F001028D
S31508008E2CC3F80022D3F8002222F47C52C3F800229D
S31508008E3CD3F80022486A42EA0022C3F800224A699B
S31508008E4C012000FA02F2D3F81C42D0430440C3F8BE
S31508008E5C1C42CB69B3B9324BD3F80C420440C3F865
S31508008E6C0C42CE688D884C6945EA0645483443F869
S31508008E7C34508E680C884D6944EA0644483503EB31
S31508008E8CC5035C60CB69012B1DD08B69002B32D1D5
S31508008E9C234CD4F804320340C4F804320B698BBB58
S31508008EAC1F4BD3F814422040C3F814020B6A012B4B
S31508008EBC2FD01B4AD2F8003223F00103C2F8003235
S31508008ECC002070BC7047164BD3F80C421443C3F8F9
S31508008EDC0C420E688D884C6945EA0645483443F8B9
S31508008EEC34508E688C894D6944EA0644483503EB40
S31508008EFCC5035C60C9E70A4CD4F804321343C4F8BA
S31508008F0C0432CBE70648D0F814321343C0F81432AF
S31508008F1CCCE70349D1F81C321A43C1F81C22C8E71E
S31508008F2C0064004038B590F82030DBB2012B05D030
S31508008F3C436A43F400234362012038BD04460223E6
S31508008F4C80F820300268136823F00103136000F0E0
S31508008F5CCBFC054623685B6813F0010F0DD000F0B7
S31508008F6CC3FC401B0A28F5D9636A43F400336362D1
S31508008F7C052384F820300120DFE700206062DCE757
S31508008F8C30B490F82040E4B2012C05D090F820407B
S31508008F9CE4B2022C40F08B8051B90468E46814F0F2
S31508008FAC030F12D1436A43F40013436201206CE0A9
S31508008FBC01290AD10468246914F0030F05D1436A00
S31508008FCC43F40013436201205FE0056801F11B04BA
S31508008FDC24012C5904F004049460002C57D105681C
S31508008FEC01F11B0424012C59640D1460056801F168
S31508008FFC1B0424012D59C5F34005D5600568254485
S3150800900C6D6805F00F051561056825446D68C5F38F
S3150800901C0725956105682C446468240C546104681A
S3150800902C0A011444D4F8B8411C7004681444D4F8E2
S3150800903CB841240A5C7004681444D4F8B841240C6A
S3150800904C9C7004681444D4F8B841240EDC70046887
S3150800905C1444D4F8BC411C7104681444D4F8BC41BB
S3150800906C240A5C7104681444D4F8BC41240C9C7121
S3150800907C04682244D2F8BC21120EDA7179B9026856
S3150800908CD36843F02003D360002030BC70470568D2
S3150800909C01F11B0424012C59E4085460A6E70129A4
S315080090ACF2D10268136943F020031361ECE7436AB3
S315080090BC43F4802343620120E7E70000074AD3689C
S315080090CC23F4E0631B041B0C000200F4E060184355
S315080090DC40F0BF6040F40030D060704700ED00E00F
S315080090EC30B4174BDB68C3F30223C3F10704042C13
S315080090FC28BF04241D1D062D01D9033B00E00023BF
S3150800910C4FF0FF3505FA04F421EA0401994005FAF3
S3150800911C03F322EA03031943002809DB0901C9B240
S3150800912C00F1604000F5614080F8001330BC7047D0
S3150800913C00F00F000901C9B2024B1954F6E700BF3B
S3150800914C00ED00E014ED00E00138B0F1807F0AD2A2
S3150800915C064B5860064AF02182F8231000209860C6
S3150800916C07221A6070470120704700BF10E000E024
S3150800917C00ED00E0042805D0054A136823F0040323
S3150800918C13607047024A136843F004031360704770
S3150800919C10E000E0704708B5FFF7FCFF08BD0000BB
S315080091AC00230F2B00F2D680F0B482B039E00722E8
S315080091BC00E00022B2403A430235674E46F82520B5
S315080091CC664A1568E24302EA05064F6817F4803FBB
S315080091DC01D044EA0506614D2E606D6802EA050663
S315080091EC4F6817F4003F01D044EA05065B4D6E60E4
S315080091FCAD6802EA05064F6817F4801F01D044EAE9
S3150800920C0506564DAE60ED682A404E6816F4001FEA
S3150800921C01D044EA0502514CE26001330F2B00F2EF
S3150800922C968001229A400C681440A242F5D14D68EA
S3150800923C022D01D0122D10D1DE08083650F826C0A2
S3150800924C03F00705AF000F25BD402CEA050C0D6988
S3150800925CBD4045EA0C0540F8265006685F00032514
S3150800926CBD40ED4305EA060C4E6806F00306BE4003
S3150800927C46EA0C0606604E6806F1FF3CBCF1010F87
S3150800928C03D9112E01D0122E10D1866805EA060CC8
S3150800929CCE68BE4046EA0C068660466826EA020296
S315080092AC4E68C6F300169E4016434660C2681540C3
S315080092BC8A68BA402A43C2604A6812F0805FACD00A
S315080092CC00220192264A556C45F480455564526C29
S315080092DC02F480420192019A9D08AE1C1E4A52F86D
S315080092EC267003F0030296000F22B24027EA020703
S315080092FC1C4A90423FF45DAF02F5806290421AD048
S3150800930C02F58062904218D002F58062904216D01F
S3150800931C02F58062904214D002F58062904212D017
S3150800932C02F58062904210D002F5806290423FF4BA
S3150800933C3EAF08223EE701223CE702223AE7032227
S3150800934C38E7042236E7052234E7062232E702B06C
S3150800935CF0BC7047704700BF00380140003C014024
S3150800936C00380240000002400AB1816170470904C6
S3150800937C816170472DE9F843044601680A6922F4AD
S3150800938C4052C36813430B610168CA6822F416423B
S3150800939C22F00C0283680069034360690343E069A1
S315080093AC03431343CB6021684A6922F44072A369CC
S315080093BC13434B61E369B3F5004F60D02368B84A91
S315080093CC934200F0148102F58062934200F00F81FB
S315080093DCFFF748FC00EB800000EB80006568AD00E9
S315080093ECB0FBF5F5AF4FA7FB05356D092E01FFF759
S315080093FC39FC00EB800000EB80006568AD00B0FB23
S3150800940CF5F9FFF72FFC00EB800000EB8000656890
S3150800941CAD00B0FBF5F5A7FB05356D094FF06408F3
S3150800942C08FB15952D013235A7FB05356D0905F099
S3150800943CF0053544FFF716FC00EB800000EB8000C6
S3150800944C6668B600B0FBF6F6FFF70CFC00EB80007E
S3150800945C00EB800063689B00B0FBF3F0A7FB0030C1
S3150800946C400908FB10684FEA081808F13208A7FBF0
S3150800947C0837C7F3431723682F449F600DE1236809
S3150800948C874A93425BD002F58062934257D0FFF726
S3150800949CE9FB00EB800000EB800065686D00B0FB13
S315080094ACF5F5804FA7FB05356D092E01FFF7DAFB9D
S315080094BC00EB800000EB800065686D00B0FBF5F9E9
S315080094CCFFF7D0FB00EB800000EB800065686D00B1
S315080094DCB0FBF5F5A7FB05356D094FF0640808FBDD
S315080094EC1595ED003235A7FB05356D096D0005F4AC
S315080094FCF8753544FFF7B6FB00EB800000EB8000EF
S3150800950C66687600B0FBF6F6FFF7ACFB00EB80005E
S3150800951C00EB800063685B00B0FBF3F3A7FB032347
S3150800952C5B0908FB13684FEAC80808F13208A7FB61
S3150800953C0837C7F3421723682F449F60ADE0FFF73F
S3150800954CA1FB00EB800000EB800065686D00B0FBAA
S3150800955CF5F5544FA7FB05356D092E01FFF792FB60
S3150800956C00EB800000EB800065686D00B0FBF5F938
S3150800957CFFF788FB00EB800000EB800065686D0048
S3150800958CB0FBF5F5A7FB05356D094FF0640808FB2C
S3150800959C1595ED003235A7FB05356D096D0005F4FB
S315080095ACF8753544FFF76EFB00EB800000EB800086
S315080095BC66687600B0FBF6F6FFF764FB00EB8000F6
S315080095CC00EB800063685B00B0FBF3F3A7FB032397
S315080095DC5B0908FB13684FEAC80808F13208A7FBB1
S315080095EC0837C7F3421723682F449F6055E0FFF7E7
S315080095FC49FB00EB800000EB80006568AD00B0FB12
S3150800960CF5F5284FA7FB05356D092E01FFF73AFB33
S3150800961C00EB800000EB80006568AD00B0FBF5F947
S3150800962CFFF730FB00EB800000EB80006568AD00AF
S3150800963CB0FBF5F5A7FB05356D094FF0640808FB7B
S3150800964C15952D013235A7FB05356D0905F0F00585
S3150800965C3544FFF717FB00EB800000EB80006668CB
S3150800966CB600B0FBF6F6FFF70DFB00EB800000EB3F
S3150800967C800063689B00B0FBF3F0A7FB0030400941
S3150800968C08FB10684FEA081808F13208A7FB0837D8
S3150800969CC7F3431723682F449F60BDE8F88300BFC0
S315080096AC001001401F85EB512DE9F04105460F4688
S315080096BC16469846069C2B681B6837EA03030CBFAC
S315080096CC01230023B3421DD1B4F1FF3FF3D02CB1D3
S315080096DC00F00AF9A0EB0800A042ECD92A68D36876
S315080096EC23F4D073D3602A68536923F001035361BA
S315080096FC202385F8393085F83A30002385F8383038
S3150800970C032000E00020BDE8F081704758B310B57F
S3150800971C044690F839300BB3242384F83930226880
S3150800972CD36823F40053D3602046FFF723FE226840
S3150800973C136923F4904313612268536923F02A03AF
S3150800974C53612268D36843F40053D3600020E06366
S3150800975C202384F8393084F83A3010BD80F8383034
S3150800976CFFF7D3FFD8E7012070472DE9F04182B007
S3150800977C1E4690F83A30DBB2202B5AD104460D46D9
S3150800978C9046002959D0002A59D090F83830012B28
S3150800979C57D0012380F838300023C363222380F87E
S315080097AC3A3000F0A1F80746A4F82C80A4F82E80CD
S315080097BC1DE000963B46002220212046FFF774FF49
S315080097CC002840D1236933B923685B68C3F30803BF
S315080097DC25F8023B0BE023685B68DBB225F8013BF6
S315080097EC05E023685B6803F07F0305F8013BE38D0E
S315080097FC9BB2BBB1E38D013B9BB2E385A368B3F582
S3150800980C805FD6D000963B46002220212046FFF7E3
S3150800981C4BFFD0B92369002BE3D123685B6805F8A5
S3150800982C013BE4E7202384F83A30002084F838001A
S3150800983C00E0022002B0BDE8F0810120FAE7012021
S3150800984CF8E70220F6E70320F4E70320F2E7000026
S3150800985C10B504460E4B18784FF47A73B3FBF0F335
S3150800986C0C4A1068B0FBF3F0FFF76EFC68B90F2CC6
S3150800987C01D901200AE0002221464FF0FF30FFF7FC
S3150800988C2FFC054B1C60002000E0012010BD00BF1A
S3150800989C300400202C0400203404002008B50B4B9F
S315080098AC1A6842F400721A601A6842F480621A60E6
S315080098BC1A6842F480721A600320FFF7FFFB002037
S315080098CCFFF7C6FF00F0D2F8002008BD003C0240A6
S315080098DC034A1168034B1B780B441360704700BF8F
S315080098EC3005002030040020014B1868704700BF73
S315080098FC3005002008B5FFF7AFF9084BA3FB00307D
S3150800990C8009FFF721FC0420FFF734FC00221146DE
S3150800991C4FF0FF30FFF7E4FB08BD00BFD34D6210D4
S3150800992C08B5FFF7E1FF08BD08B5FFF7D1FFFFF74C
S3150800993C32FC08BD08B501224FF480510148FFF7E7
S3150800994C13FD08BD0008024010B5FFF7E9FF104BE0
S3150800995C1B68C31AB3F5FA7F0ED304460D4B1B7856
S3150800996C5BB90C4B01221A7000224FF480510A483D
S3150800997CFFF7FAFC064B1C6010BD064B00221A704A
S3150800998C01224FF480510448FFF7EEFCF2E700BFC2
S3150800999C580400205404002000080240014A024BD7
S315080099AC9A6070470080000800ED00E000B595B09D
S315080099BC00210191204B1A6C42F080521A641B6CE0
S315080099CC03F080530193019B02911C4B1A6842F4D5
S315080099DC80421A601B6803F480430293029B01239E
S315080099EC08934FF48033099302230E934FF48002A5
S315080099FC0F92082210924FF4A87211921293072311
S31508009A0C139308A8FEF744FE00B1FEE70F23039351
S31508009A1C02230493002305934FF4A05306934FF4A3
S31508009A2C80530793052103A8FFF768F800B1FEE7F2
S31508009A3C15B05DF804FB00BF00380240007000400A
S31508009A4C08B5FFF7ABFFFFF729FFFFF7AFFFFFF7E7
S31508009A5C51FFFFF76FFF08BD08B5FFF7F1FF00F0E0
S31508009A6C53F9FFF771FF00F0D3F9FAE770B58CB02C
S31508009A7C002400944C4B5A6C42F480425A645A6C3B
S31508009A8C02F480420092009A01941A6C42F08052B9
S31508009A9C1A641A6C02F080520192019A02941A6B9B
S31508009AAC42F001021A631A6B02F001020292029A40
S31508009ABC03941A6B42F002021A631A6B02F0020242
S31508009ACC0392039A04941A6B42F004021A631A6BF3
S31508009ADC02F004020492049A05941A6C42F40032B9
S31508009AEC1A641A6C02F400320592059A06941A6CDA
S31508009AFC42F000721A641B6C03F000730693069B03
S31508009B0C0320FFF7DBFA224621466FF00B00FFF71E
S31508009B1CE7FA224621466FF00A00FFF7E1FA2246D9
S31508009B2C21466FF00900FFF7DBFA224621466FF053
S31508009B3C0400FFF7D5FA224621466FF00300FFF71B
S31508009B4CCFFA224621466FF00100FFF7C9FA2246E2
S31508009B5C21464FF0FF30FFF7C3FA4FF480530793B3
S31508009B6C0125089509940A9407A91048FFF718FBCC
S31508009B7C0C23079302260896099503250A950723AD
S31508009B8C0B9307A90A48FFF70BFB4FF4407307938F
S31508009B9C089609940A9509230B9307A90548FFF714
S31508009BACFFFA0CB070BD00BF003802400008024036
S31508009BBC000002400004024008B50848084B036040
S31508009BCC4FF46143436000238360C3600361836180
S31508009BDC0C224261C361FFF799FD08BD840400207D
S31508009BEC004400402DE9F04104460D4617469846B8
S31508009BFCFFF738F8154BA3FB00308009002201E06B
S31508009C0C0132D2B2112A1DD8114B13F8121003EBDC
S31508009C1C420393F801C001EB0C0303FB0443B0FBAE
S31508009C2CF3FE03FB1E06002EEAD11FFA8EF32B80D9
S31508009C3C013B9BB2B3F5806FE2D2397088F800C04D
S31508009C4C012000E00020BDE8F08100BFD34D621072
S31508009C5C5C9E000830B58DB00025ADF82E508DF8F9
S31508009C6C2D508DF82C500BAB0DF12D020DF12E014C
S31508009C7C4FF4FA70FFF7B6FF1A4C1B4B2360257688
S31508009C8C6576A576E57625776577A560E5609DF812
S31508009C9C2D30013B1B0423619DF82C30013B1B0521
S31508009CAC6361BDF82E3063602046FEF7FCFF06950F
S31508009CBC0795012308934CF6E042019202954FF65C
S31508009CCCE072039204220492059509930E230A93D3
S31508009CDC0DEB02012046FFF78DF82046FFF722F917
S31508009CEC0DB030BD5C0400200064004008B50023AC
S31508009CFC012201460348FFF738FD08B1002008BDCC
S31508009D0C0120FCE78404002008B5FFF755FFFFF790
S31508009D1CA1FF08BDBFF34F8F0549CA6802F4E0627C
S31508009D2C044B1343CB60BFF34F8F00BFFDE700BF57
S31508009D3C00ED00E00400FA0508B5214B1B78B3B911
S31508009D4C2048FFF7D3FF012800D008BD1D4B1B7810
S31508009D5C013BDBB23F2BF8D8FFF7E2FD1A4B186034
S31508009D6C174B01221A70194B00221A70EDE7174B84
S31508009D7C1B78013313481844FFF7B8FF012813D191
S31508009D8C124A13780133DBB213700E4A12789342D7
S31508009D9CDBD10B4A002111700A4A5278FF2AD4D11A
S31508009DAC022BD2D1FFF7B6FFFFF7BAFD064B1B689D
S31508009DBC64339842C9D9024B00221A70C5E700BF12
S31508009DCC05050020C404002008050020060500200F
S31508009DDC00B58BB001AB03AA00210C48FFF7D0F8ED
S31508009DEC20B9039A40F267639A4202D00BB05DF829
S31508009DFC04FB059B002BF9D19DF80430FF2BF5D1FC
S31508009E0C079B022BF2D1FFF785FF00BF5C040020ED
S31508009E1C08B5FFF791FFFFF7DBFF08BDF8B500BFE4
S31508009E2CF8BC08BC9E467047F8B500BFF8BC08BC21
S30908009E3C9E46704779
S31508009E4000000020000000000000000001020304DA
S31508009E5006070809000000000102030405020602BD
S31508009E60060307030803090309040A040B040C0480
S31508009E700C050D050E050F050F0610061007100830
S30D08009E807CE3FF7F01000000EE
S30D08009E8819850008B1810008E4
S30908009E908D810008AA
S31508009E9400000000EC02002054030020BC0300204C
S31508009EA400000000000000000000000000000000A0
S31508009EB40000000000000000000000000000000090
S31508009EC40000000000000000000000000000000080
S31508009ED40000000000000000000000000000000070
S31508009EE40000000000000000000000000000000060
S31508009EF40000000000000000000000000000000050
S31508009F04000000000000000000000000000000003F
S31508009F14000000000000000000000000000000002F
S31508009F24000000000000000000000000000000001F
S31508009F34000000000000000001000000000000000E
S31508009F440E33CDAB34126DE6ECDE05000B000000D3
S31508009F5400000000000000000000000000000000EF
S31508009F6400000000000000000000000000000000DF
S31508009F7400000000000000000000000000000000CF
S31508009F8400000000000000000000000000000000BF
S3150800A2B400000000000000000C0500200024F40043
S30D0800A2C4010000001000000073
S705080085FD70
